:10000000A0019D2990002408840022081021841357
:100010000005181C2206031920281008031D1828A3
:100020001608FF3E031C21280A3025211608212826
:10003000100AFF3003192028100B20281708212848
:1000400099090310191803149829A016A01EA012CC
:1000500020192E28A100201503109829201A3628CF
:10006000920020164D2003183B2812085420031834
:100070003B28A01E982946206B2020112012A01199
:10008000240884002208841780044C282408840053
:100090002209800584178005080040206B20462037
:1000A00067202108A01901388E0008308F008E0DBE
:1000B00003184020031C46206B2067208F0B572815
:1000C00040206B202408840022080005FF3E2508FC
:1000D0008400230949282508840023088004841704
:1000E000230980054C2891019000A11727308F002B
:1000F0001030862003308F00E83086208F01643076
:1001000086208F010A308620100891288E00110861
:100110008D0010088C0061210C08031DA113A11B88
:100120000800303E94280408A018BF2893008611C8
:100130008316861183123A308D0098303321861051
:100140008316861083123330920083160F30860593
:100150008312D3200F308D00DC303321D3203C308C
:100160003221D32022309200D3202030BE200C3008
:10017000BE200630BE20A0141308BF282014920011
:10018000201CCD288610033C031CD228D2203E30F0
:100190008D0080303321031408002014FE3C031925
:1001A00098298614201C20100F3086051208F0397B
:1001B00086048615920E86112018D3282830322105
:1001C00003140800A11315080319A11705309400A2
:1001D00027308F001030F82003308F00E830F820EF
:1001E0008F016430F8208F010A30F8201008FF28B2
:1001F0008E0011088D0010088C0061210C088C0005
:1002000094030319A11315080319092914020318EB
:1002100008000C08031DA113A11B0800303E932900
:10022000841780049829890083160814831208080B
:10023000982988008316081555308900AA3089004E
:10024000881488182129081198298F018E00FF3001
:100250008E07031C8F07031C982903308D00DF30A5
:10026000332127298D01E83E8C008D09FC30031CC9
:100270003C298C07031839298C0764008D0F392914
:100280000C1842298C1C46290000462908008E00C3
:10029000023051298E00063051298F018E00043022
:1002A000512994000F080D02031D58290E080C0255
:1002B000043003180130031902301405031DFF3008
:1002C000982910309200910190010D0D900D910D23
:1002D0000E0890020F08031C0F0F910203187729D4
:1002E0000E0890070F0803180F0F910703108C0DCD
:1002F0008D0D920B65290C089829103094008D0102
:100300008C01930C920C031C8B290E088C070F0890
:1003100003180F0F8D078D0C8C0C910C900C940B07
:1003200081291008982984001D088A001C08820071
:1003300083130313831264000800831605148514C5
:100340000515051685158312C230B6004030AE0083
:100350001F30AF000130BD00643025210611831627
:100360000611FE30831294200130942052309420E4
:100370005830942020309420313094202E30942016
:100380003230942047309420483094207A309420A2
:1003900020309420203094207630942032309420E5
:1003A0002E30942035309420BE0103308F00E83089
:1003B00026213E081321B20001303E079E009F0116
:1003C0009F0D1E081321B3002E083207AC002F0822
:1003D0000318013E3307AD00FC302C07B0000E308F
:1003E0000318013E2D07B1000630A4000130A20021
:1003F0000630A5000230A300360827203108272048
:10040000300827208E302520B522E02201308F00D1
:10041000F43026210530A4000830A2009801FF30F6
:1004200096009701013099003B080220BB00031899
:100430006A2A0530A4000830A20001309800FF307D
:1004400096009701013099003C080220BC00031877
:100450006F2A0530A4000130A20098010A309600EE
:10046000023097000130990037080220B7000318C6
:10047000752A0530A4000230A20098010A309600C7
:10048000023097000130990038080220B8000318A4
:10049000862A0530A4000430A2009801FF3096009F
:1004A0009701013099003A080220BA000318382B4E
:1004B0000530A4001030A2009801FF30960097018B
:1004C0000130990039080220B9000318A42A6430C9
:1004D00025210A2ABE014130B400B501D9290230D4
:1004E000BE004230B400B501D9293D08B207031857
:1004F000B30A32088C0033088D0012308F00C030F0
:100500004A21031D852AB201B301E42932088C0077
:1005100033088D003D084D21031DA12A32088C00AF
:1005200033088D008F0100304721031D9C2A3D08B0
:10053000B202031CB303E429C030B2001230B3008E
:10054000E429B201B301E42964003D08083C031921
:10055000AF2A0310BD0D0B23B522E0220A2A013079
:10056000BD000B23B522E0220A2A40302C02A6004F
:100570001F30031C013E2D02A70026088C0027080F
:100580008D0008308E008F016121A8000D08A900A0
:1005900026088C0027088D0008308E008F0161210D
:1005A00010089E0011089F007D30920093011E08E4
:1005B0008E001F088F007D21AA001108AB000800E3
:1005C000FE309420013094200130732003309500D8
:1005D000280890002908910093309C009D01E2209A
:1005E0002E309420033095002A0890002B089100AB
:1005F00093309C009D01E220203094204D309420C7
:10060000483094207A309420203094202030942058
:10061000340894200800FE3094200130942050309B
:1006200094206130942073309420203094206430E2
:10063000942065309420203094207D3092009301E6
:100640003D088E008F017D219E0011089F001F082C
:1006500091001E087420203094206B309420483084
:1006600094207A30942005308F00DC302621080059
:100670003E0889003208192101303E079E009F0183
:0C0680009F0D1E088900330819210A2A6A
:02400E00F53F7C
:08420000D4000800E0000100F9
:00000001FF
